:020000001028C6
:02000800492885
:10002000FF309A009B009B0B13289A0B1328850125
:1000300086018316850105150516860106148614AA
:10004000061601178116011281110110811001118C
:1000500083120B160730990064309C0005080439A0
:1000600013069500151D2E28050804399300131951
:100070004228181C3D2818102E2881010B118B10C6
:100080008B172E289C0B2E288B13492064309C0044
:100090002E289700030E9600831601158114011473
:1000A0008312990B5928073099008615000000002B
:1000B000861100308C008D008E000B1D66280230EA
:1000C0008C0005308D0006308E000B11811F6F28CB
:1000D00001308F000230900008309100AF20011FE6
:1000E000782800308F000630900004309100AF2057
:1000F000811E812800308F00033090000230910073
:10010000AF20011E8A2800308F0001309000063099
:100110009100AF20811D932800308F0000309000A7
:1001200008309100AF20011D9C2800308F00003066
:10013000900004309100AF20811CA52800308F0072
:100140000030900002309100AF20011CC828003020
:100150008F000030900001309100AF20C8280301CB
:100160000E0711078E00F63E031CB9288D0A0A30CF
:100170008E0203010D0710078D00F63E031CC328F5
:100180008C0A0A308D0203010C070F078C0008004F
:100190008C1CD4280C1CD4280D1DD4288D1CD428CC
:1001A0008C018D018E01D42830308E048D048C0496
:1001B000D9281D18DC28E3288612432186164321FE
:1001C00002309D0049298618F3289E0A9E18492965
:1001D0009E19492909309F00A000A10000309E000F
:1001E00001309D00492901309D0000309E004321CF
:1001F000061143219F01A001A1012A212A212A21C0
:100200002A212A212A212A219F002A219F0D1F10FD
:100210009F042A21A00D2010A0042A21A00D201047
:10022000A0042A21A00D2010A0042A21A00D201036
:10023000A0042A21A10D2110A1042A21A10D211021
:10024000A1042A21A10D2110A1042A21A10D211010
:10025000A10440290F30A200A20B2C2906130F3055
:10026000A200A20B312906170000000000000608BA
:10027000A300A30CA30CA30CA30C230801390800B2
:100280000615432149291030A400A721A40B4529B4
:1002900008003030A104A0049F044E2925309200AC
:1002A0007C210C0892007C210D0892007C210E0814
:1002B00092007C212F3092007C21373092007C21EB
:1002C0002F3092007C211F0892007C212008920090
:1002D0007C21210892007C210D3092007C21181491
:1002E00064309C0083160111811001108312160ED8
:1002F0008300970E170E0800A121121CA1211218CD
:10030000A421921CA1219218A421121DA12112192D
:10031000A421921DA1219219A421121EA121121A19
:10032000A421921EA121921AA421121FA121121B05
:10033000A421921FA121921BA421A121A421A421C7
:1003400008008511A72108008515A7210800ED30B8
:080350009400940BA929080098
:00000001FF
